:020000040000FA
:020000000E28C8
:080008008B13A000030EA10000
:100010008B10210E8300A00E200E09008B130B13F2
:100020008B120B168B110B118B100B108501860197
:100030008316F0308500FF3086000117811681118C
:100040000114811401158312842084202E200000C5
:10005000000000008B1763008B13242881016F20A0
:100060000108A5002508023C031837283A2800306B
:10007000A6006C282508053C03183F2842280430B8
:10008000A6006C2825080A3C031847284A28023095
:10009000A6006C282508143C03184F285228063067
:1000A000A6006C282508293C031857285A28013037
:1000B000A6006C2825084C3C03185F2862280530F0
:1000C000A6006C282508703C031867286A280330AE
:1000D000A6006C280730A6002608850008006E30B0
:1000E000A200000000000000000000000000A20BC1
:1000F00071282330A2000000000000000000000072
:100100000000A20B7B2808006430A3006E30A4001E
:10011000000000000000000000000000A40B882880
:06012000A30B8628080075
:02400E00F13F80
:00000001FF
